:030000000219FDE5
:03000B000200A848
:03002B0002018847
:03005B0002033C61
:030073000203295C
:1000800002030406080C10182030406080040608A3
:100090000C10182030406080A0C00003070F1F051F
:1000A000050D050305030302C2AF306308C2638573
:1000B000798AD2AF32C0D0C0E0206221E525601637
:1000C000E473E525F4C3334009758A00D263F579FA
:1000D00001D4F58AD262D0E0D0D0D2AF32C3E526C7
:1000E000334009758A00D263F57901EEF58AC26260
:1000F000E526F4603030682620720DD0E0D0D0C202
:1001000095C294C293D2AF32C295C294C293206F6B
:100110000D20660A7414D5E0FDE57BF45290D0E022
:10012000D0D0D2AF32758A00D263757900C28DD239
:1001300062211E01C2306805206602D29501C230DC
:100140006805206602D29401C2306805206602D29A
:100150009301C2D29230680A2066077410D5E0FD80
:10016000D29501C2D29130680A2066077410D5E09A
:10017000FDD29401C2D290D29230680A20660774F0
:1001800010D5E0FDD29301C2C2AFC2AD53E6EFC0BD
:10019000D0C0E0D2D3D2AFE57A6009E577600575CB
:1001A000770041D6757701C2CEE52A6007207449F1
:1001B000152A21F97800790020742EE580307E011F
:1001C000F430E70278FF53DACF207E0343DA2030A1
:1001D0007E0343DA10C2D8C271E580307E01F4306C
:1001E000E70279FFC3E89970CB306103752A1820C4
:1001F0007403752A18885CD27020740DE52B600496
:10020000152B410943DA01C2D8207002417CA85C59
:10021000206102C270207431C3E894F0400374F08E
:10022000F8E8C4540F28F87984B703024149C3138E
:10023000C3138721200802C313200A06C3C898F8F5
:10024000414928F8500374FFF8C3E895655003E569
:1002500065F88822E52D54066022206B1FE536C321
:1002600033C333F8E564C313C313F9C395224002C3
:100270008922E82522F52250037522FF852224A831
:1002800024C3E52495614002A8618825E5667002D3
:1002900041C0C3E8AA669A5003E8FAE4F9EAC33316
:1002A000FBE568F45B29400D2567F8E567600215FA
:1002B00067400B41C00AC3E5679A5002056778FFA3
:1002C0008826C26FC3E52694F84002D26FC3E525A5
:1002D00094404002D26420CF0AD0E0D0D043E61050
:1002E000D2AD32C2CF053AE57A6009E5786005758E
:1002F0007800611F7578017801E52A600530740285
:10030000152AC3E55C94014005755F00611F7560A7
:1003100000756900E55F2401F55F5003755FFFD04C
:10032000E0D0D043E610D2AD32C2AF53E67F759233
:10033000FA7593FFC260759104D2AF32C2AF53E633
:10034000EFC2ADC0D0C0E0C0F0D2D3D2AFA8FBA9FD
:10035000FCE57A6007C3E913F9E813F8C2D83071F5
:100360000261AE53DACF207E0343DA10307E0343BE
:10037000DA20D271E580307E01F420E702618588C1
:10038000278928A1DB53DACF207E0343DA20307E91
:100390000343DA10C2D8C271307402A1C77800E5F5
:1003A00080307E01F430E702A1C7885CA1AF53DA48
:1003B000CF207E0343DA20307E0343DA10C271205F
:1003C0006102818753DACF207E0343DA10307E0347
:1003D00043DA20C2D8D27188578958C3E89555F8B6
:1003E000E99556F97B007E087A00C3E8948CE9947D
:1003F000005005755B008179882178A2E6A821600C
:1004000055C3E894C8E994005008E4D2E4FB7A0AA2
:100410008154C3E89468E994015008E4D2E3FB7A7C
:100420000F8154C3E894D0E994025008E4D2E2FB6F
:100430007A1E8154C3E894A0E994055008E4D2E1FF
:10044000FB7A3C8154C3E89498E994085008E4D2BC
:10045000E0FB7A787E00C3E89559FCE9955AFD30B7
:10046000E70AECF42401FCEDF43400FD755B00C3F5
:0D047000EC9AED9E5003755B018859895A86
:10047D008557558558567802A1AFC3E89527F8E9F9
:10048D009528F9307C02A193307B02A193307A023A
:10049D00A18C20750281AAE9FDE8FC81C9E9C3138D
:1004AD00F9E813F8307902A18CE9C313F9E813F8D0
:1004BD00307802A18CE9C313FDE813FC20612CC335
:1004CD00EC941CED9402400281E0ED701EC3EC949F
:1004DD00C850180529E52970021529C3E529940A84
:1004ED005002A1C7755C00D270A1C7E52960021545
:1004FD00297888E6F97400207F087896B903027888
:10050D009EE624FAFEE43400FFC3EC9EFCED9FFD55
:10051D009208B90310A2085007207609D276A132AD
:10052D00307602C276A2085016B9030DECF4240100
:10053D00FCEDF43400FD02054C78007900A193B96F
:10054D000315EC33FCED33FDC3EC940AFCED940084
:10055D00FD50047C007D00C3EC94FFED940040063B
:10056D0078FF7900A193EC8572F0A4C5F0A2F73362
:10057D00F8790040030205AF78FF79000205AFE975
:10058D00C313F9E813F8307C0EE9600278FFC3E875
:10059D001338F8E43400F9C3E894FFE994004002FD
:1005AD0078FF885CD270206102A1C7741FF4552FAB
:1005BD004BF52FC274EB7002D274752A1830740388
:1005CD00752A0A306102A1DB20740353DAFE207410
:1005DD0003752B06D0F0D0E0D0D0D2AD43E610326B
:1005ED00790102060B790302060B790A02060B79D3
:1005FD001E02060B796402060B79C802060B7817EA
:10060D00E4D5E0FDD8FAD9F6227A147B78020632C9
:10061D007A107B8C0206327A0D7BB40206327A0B8D
:10062D007BC80206327902E4D291D5E0FDD294D591
:10063D00E0FDC294D5E0FDC291D5E0FDE920E002D8
:10064D00D29530E002D293E573D5E0FDE920E002CA
:10065D00C29530E002C2937496D5E0FDD9C9EAF88F
:10066D00D5E0FDD8FBDBBED29122C37C007D0075A9
:10067D00F00005F0EA33FAEB33FB50F6EB13FBEA2F
:10068D0013FAC3E9FFE8FEE89AF8E99BF95004EF85
:10069D00F9EEF8B3EC33FCED33FDD5F0DFEDF9EC0D
:1006AD00F822E889F08A20D2D4F8A9F07B0030F73F
:1006BD000B7BFFF42401F8E9F43400F9E88520F010
:1006CD00A4ADF0F8E98520F0A4AFF0FEED2EF9749D
:1006DD00003FFA7C04C3EA13FAE913F9E813F8DCD6
:1006ED00F48BF030F70AE8F42401F8E9F43400F95A
:1006FD00E889F0C2D4F8A9F02222C3E54113F9E547
:10070D004013F8C3E54498F8E54599F9500CC3E852
:10071D009480E994FF401602073EC3E8947FE99464
:10072D0000500302073E787F790002073E788079FA
:10073D00FF8849894A22E5492546F8E54A3547F9B2
:10074D00854A20E4300701F43548FA30E709C3EA59
:10075D0094F0401502077CC3EA940F500302077C06
:10076D0078FF79FF7A0F02077C780079007AF0C361
:10077D00E5249561500AC374019524500B02079A24
:10078D00E54A20E70E02079AE54A30E706884689D2
:10079D00478A482278A5E6FAC3E54933F8E54A3396
:1007AD00F9D1AFE930E70BC3E89480E994FF40132A
:1007BD00E1D4C3E8947FE994005002E1D4787F79C5
:1007CD0000E1D4788079FFE820E715C3E52398F898
:1007DD004009C3E8940140030207FB78010207FBBF
:1007ED00E8F424012523F840030207FB78FF884B2A
:1007FD002278A6E6FAA847A9481206AFE930E70C19
:10080D00C3E89401E994FF4016020830C3E894FF51
:10081D00E99400500302083078FF7900020830781F
:10082D000179FFE920E715C3E54B98F84009C3E8C6
:10083D00940140030208577801020857E8F4240197
:10084D00254BF8400302085778FF88242278FFC211
:10085D006420693D206A12D264C3E541940A4009BF
:0E086D00C3E52594405002C26479A1E76023E0
:10087B00E541601F74FF8541F0848539F0306A03D0
:10088B0075F005A4F8C5F0600278FFC3E8956450D5
:10089B0002A864886322C3E54094C8E5419400E54F
:1008AB006350031401B2046002F563220208BA22FA
:1008BB0075E890227883E6FFE5E820ECF7A8BDA960
:1008CB00BE0570C3E57094084052757000E9FA7963
:1008DB00A0E76044EA7007E571601B0208F5C3E806
:1008EB0095716010E5715006600C140209010460EB
:1008FB00F9020901E571F571C39472401B7561C072
:10090B00C394044013756180C39404400B7561401C
:10091B00C39404400375610075BB0622E561F46066
:10092B00020561E570B4070375BB1022743279A719
:10093B0087F0A4C5F0A2F733F8C3E895614002A88D
:10094B006188228824882588268864227540007552
:10095B0041F022C2AF75C820A8CCA9CDAA3A30CF9E
:10096B00010A75C824D2AFC3EA13FAE913F9E813E5
:10097B00F8AB3BAC3C883B893CC3E89BF8E99C203B
:10098B00690A547FF9306702417821D5AD3D8A3D24
:10099B00F9EA9D547FFA600478FF79FFAE3EAF3FD2
:1009AB008B3E8C3FA83BA93CC3E89EF8E99FF9C35B
:1009BB00E54113FBE54013FAE82AF540E93BF54125
:1009CB0050067540FF7541FF411FAA40AB41AC403B
:1009DB00AD417E047F02C3EB940440021E1FC3EBA8
:1009EB00940840021E1FC3ED13FDEC13FCDEF7C38E
:1009FB00EA9CFAEB9DFBEF6009C3E913F9E813F8E6
:100A0B00DFF7EA28FAEB39FB8A408B4150067BFF74
:100A1B008B408B41C3EB94025002D2673069047F49
:100A2B0003414A7892E6FFC3E537948240110FC326
:100A3B00E53794A040010FC3EF940640027F057E7B
:100A4B0002E541C4540FF9E541C454F0F8E540C444
:100A5B00540F28F8C3E89EFAE99400FB4009C3EA57
:100A6B009402EB940050047A02E4FB41C4AA40AB1D
:100A7B0041EBC4FEEAC4540F4EFCC3EA9CFAEB9460
:100A8B0000FBC3E813C313F8EA28FAEB3400FB8A24
:100A9B00408B41C3EB94024002C2677802EBC4FE69
:100AAB007B00EAC4540F4EFAC3EA98FA4005C3948C
:100ABB000250027A027892E6FF30600241C48551FF
:100ACB0092855293D26043E680C3E49AF8E49BF993
:100ADB00C3E833F8E933F93067026157E8FAE9FB09
:100AEB00D3E913FDE813FC88518952C3EF940360DB
:100AFB0038EF20E00DE82CF8E93DF9ECFAEDFB02BC
:100B0B000B20E828F8E939F9C3E82402F8E93400A6
:100B1B00F97AFE7BFFC3EF9403400E8A538B548804
:100B2B004D894E8C4F8D50618B885389548A4D8BD8
:100B3B004E8C4F8D503069127553F07554FF754FB5
:100B4B00F07550FF7551F07552FF618BE8FAD3E8E1
:100B5B0013FC8851C3EF94036020EF20E007E82CCF
:100B6B00F8ECFA6177E8282402F87AFEC3EF9403D5
:100B7B0040088A53884D8C4F618B88538A4D8C4F1C
:100B8B00E568C3335002646BF5683060026195759C
:100B9B003402D26043E680E52D5406602DA840A9AF
:100BAB0041C3E913F9E813F8306904E92440F9C2A9
:100BBB00AF53E67F759100C3E498F594E499F595EE
:100BCB00759104D26043E680D2AF22D265754300A3
:100BDB00752000306C03752040020BF5D265754310
:100BEB0000752040306C0375200078017901206777
:100BFB0020E52D54066002C2657914E541C31370DC
:100C0B000104F8C3941440027814306904781B79FA
:100C1B001BC3E833F8C3E933F9206010E543600CDC
:100C2B00306903D53404D26D81AC719D0543E59BCE
:100C3B005440B52002819630690908C3E8994001F8
:100C4B0018812420650A08C3E899400261F58124C4
:100C5B00C265C2AF53E67F75910030671275940081
:0F0C6B007595FC759104D26043E680D2AF61F5B8
:100C7A00AE40AF41C3EE33FEEF33FF50047EFF7F39
:100C8A00FFC3E49EF594E49FF595816EC3E5339422
:100C9A0001500261F530650261F5D80281AA81240A
:100CAA00C26DC2AF53E67F75910085539485549502
:100CBA00759104854D92854E93D26043E680D2AFFA
:100CCA00E52D54066008206A020533020CE8306DEF
:100CDA000D206C0A20650715811581021595227869
:100CEA00003064053065027801E53775F007A4F92C
:100CFA00E5F028F5F0E9A2F013A2F113A2F213F538
:100D0A0037C394785003753778C3E5379538400868
:100D1A00D266C295C294C293306002A122854F92D4
:100D2A00855093D26043E68022207D16C2AF754279
:100D3A0002D291C292306202D293D2AF759F11024F
:100D4A000F2AC2AF754202D291C290306202D29586
:100D5A00D2AF759F11020F2A307245207D22C2AF91
:100D6A00754203900164757B02C293D290D292308D
:100D7A006204D294A182C291D2AF759F01020F2A56
:100D8A00C2AF754203900164757B02C295D292305C
:100D9A006204D294A1A2C291D2AF759F21020F2AF6
:100DAA00207D17C2AF75420390013FC293306202A1
:100DBA00D294D2AF759F01020F2AC2AF7542039037
:100DCA00013FC295306202D294D2AF759F21020FC1
:100DDA002A207D16C2AF754204D292C290306202B6
:100DEA00D294D2AF759F21020F2AC2AF754204D2A4
:100DFA0090D292C292306202D294D2AF759F01020F
:100E0A000F2A307243207D20C2AF754205900153EC
:100E1A00757B04C294D291306204D295C12AC292DF
:100E2A00D2AF759F11020F2AC2AF754205900175A4
:100E3A00757B01C294D291306204D293C14AC290A6
:100E4A00D2AF759F11020F2A207D17C2AF754205D6
:100E5A00900135C294306202D295D2AF759F1102C9
:100E6A000F2AC2AF754205900149C2943062EBD293
:100E7A0093D2AF759F11020F2A207D18C2AF754217
:100E8A0006D290D292C291306202D295D2AF759FA9
:100E9A0001020F2AC2AF754206D292C29130620293
:100EAA00D293D2AF759F21020F2A307245207D203E
:100EBA00C2AF754201900175757B01C295D292301D
:100ECA006204D293C1D2C290D2AF759F21020F2A77
:100EDA00C2AF754201900153757B04C293D290D27E
:100EEA0092306204D295C1F4C292D2AF759F0102C8
:100EFA000F2A207D17C2AF754201900149C2953071
:100F0A006202D293D2AF759F21020F2AC2AF7542F5
:100F1A0001900135C293306202D295D2AF759F011A
:100F2A00C26622900133757B00C295C294C293D2E5
:100F3A0092D291D290C26222788076FF0876FF0818
:100F4A0076FF0876FF08760308760408760A08769C
:100F5A0003087601087601788C76010876FF087610
:100F6A00FF0876FF0876FF0876FF0876030876FF03
:100F7A000876FF0876FF0876250876D00876FA08FC
:100F8A0076FA0876040876FF08760108760008766D
:100F9A007A0876FF08760108760108760008760353
:100FAA00087600227887E6FFC272BF0302D27278FF
:100FBA0088E6C394036008C27DE630E102D27DC2AE
:100FCA007E7889E630E102D27EC3EF94026008752A
:100FDA008E01D273020FE6758E00C273227880E604
:100FEA00149000809378A5F67881E6149000809397
:100FFA0078A6F67886E61490008D9378A7F6788618
:10100A00E6F539C394025003753902789CE67538BF
:10101A00FFB402037538A0B4030375388278A3E6D7
:10102A001490009A93F566120F2D22227896E6FA0A
:10103A007897E6FB7888E6B40305C3EB940EFB3099
:10104A007F047A007BFFC3EB9AFCC3948250027C34
:10105A00827572000572EC8572F0A4C3E5F0947D86
:0E106A0040F222D27F11361205FC7A007B0084
:101078007C101205F2E55C2AFA74003BFBDCF37C79
:1010880004C3EB13FBEA13FADCF7FEC27F11362226
:10109800E5EF20E6037520000520903FFFE52014CA
:1010A8006006901FFF1460009304600375EF1253ED
:1010B800D9BF7581C043FF801205ED75EF0243B2B9
:1010C80003E5B3240220E70DF521E5E320E00685DA
:1010D80021B343E301120F2D7580FF75A40075F14C
:1010E8009075D47F75908775A5BF75F2BF75D500CB
:1010F80075A60175E241120F2DE4F8F6D8FD756862
:1011080001120F421215EF78988673753001C2AF3D
:101118001206061206161205FC12061D1205FC120E
:1011280006241205FC1217081206061206061206F5
:1011380001C2AF78FA79FA308707D9FBD8F7021CD1
:1011480000120FAE120FE711351136789886731218
:101158000F2D75A90075B680757A00758810758988
:101168000275C82475910475D84075A82275B8020F
:1011780075E690759B80759D0075D10E75BC587588
:10118800BB0675BA1175E8801205EDD2AF1208B723
:1011980075360053DACF207E0343DA20307E0343CE
:1011A800DA1043DA01C2D8C271120606D2617B0393
:1011B8007A0CE55B70077A0CDB030211391205FC27
:1011C800207003021139C270E55CC3940240E1E566
:1011D8002F541F855E5DF55EB55DD5DAD5C26153C6
:1011E800DACF207E0343DA20307E0343DA10C2D8F8
:1011F800C27178A2E67008D274E52F54E0F52FC2C8
:1012080075752900120601307409C3E529940A404E
:1012180002D2751205F278023074027800C3E55CD8
:101228009840F0C2AF120616120616120616D2AF72
:10123800120606754C007888E6B40302611C120594
:10124800F2788CE6C39401500302131CE530C39472
:1012580001500302131C207435C3E55C94FF50034E
:1012680002131CC2AF12062BD2AF120601C3E55CF3
:10127800940150EFC2AF1206161205F7120616D2E5
:10128800AF120601C3E55C94FF40E902178D7F05A4
:10129800D27F1136120601C2AFC27F1136AE5CC3CF
:1012A800E55C947FD2AF40761205EDC2AF12062BF3
:1012B800D2AFDFDC116DC3EE94057897F6120606FF
:1012C8001216311217107F0AD27F1136120601C288
:1012D800AFC27F1136AE5CC3E55C947FD2AF50E6F7
:1012E8001205EDC2AF1206161205F7120616D2AF96
:1012F800DFD6116DEE24037896F612060612163123
:1013080012173F1206011136C3E55C94FF500241E3
:101318005E02178DC3E55C954C4003855C4C120654
:101328000178017988E7B403027805C3E55C984041
:1013380002413EC2AF12062B12062B12062BD2AF69
:10134800120606753000E4F531F5320531E531F461
:10135800703F0532789AE678191460127832146072
:101368000D787D14600878FA146003753200C3E5BF
:101378003298401D120F2D1205ED15327531007887
:10138800998673C2AF12062BD2AF7898867312066D
:10139800011205F7E52A7005307402213978012019
:1013A80074027806C3E55C9840A17888E6C3940384
:1013B8006003120601E52A7003021139C2AF120F49
:1013C8002DE4F522F523F524F525F526F567D2AFAA
:1013D8007885E6C333F565E4F544F545F546F54704
:1013E800F548F570F52CF52DF53775700875BB10B7
:1013F8001205ED1208BBE5E820ECFBA8BDA9BEE983
:101408007001F888711208BF75700875BB10120F4B
:10141800AEC2AF7561FF12093785226185226285E8
:101428002263D2AF75220175240175250175260145
:10143800856069756A0175B69075A903757A017832
:1014480088E6B40307C27D307602D27DD268D269BD
:10145800753300120E83120EB412095712095E1268
:0E146800095712095E120957120BE712070608
:10147600120CE9120D3312095E120BD6306E0312EE
:10148600070720670312085A3067031208A1120CD7
:10149600E9120D6212095E120BE7306E0312074362
:1014A600120CE9120DDB12095E120BD6306E031216
:1014B60007A1120CE9120E0C12095E120BE7306E30
:1014C600031207FE120CE9120E8312095E1208BB04
:1014D600120BD6120CE9120EB41208BF12095E30B6
:1014E600692F856461856462856069756A0179180A
:1014F6007A0CC3E53399400CC269D26A8A357561A4
:10150600FF021517C3E55C9401400302147002152F
:101516009D306A1D206C1AE535147006C26AD26BBE
:101526008170F535C3E55C94014003021470021521
:101536009D753600788279A4E760027803C3E55F7B
:10154600985054307404E52A604D7888E6B4031741
:10155600207D05207607A16D307602A16D206C07EF
:10156600D26C85646181AF78F0306C0585646178F2
:1015760020C3E5419850028170306C1BC26CC27D5D
:10158600307602D27DD26A75351285646181700526
:1015960036E55C6002A1A0753600C2AF120F2D7849
:1015A60087E6FE7602120FAE7887EEF6E4F522F5B0
:1015B60023F524F525F526F565752C00752D0075A2
:1015C600A90075B680757A00D2AF120601120F2DEA
:1015D60078A4E66006C292C291C290307409C3E54F
:1015E60036940440022139614E901A0D7820121665
:1015F60073E520B45A0CA3121673E520B4A50302B2
:101606001611120F42121631021630901A03788004
:101616007B0A121673A308DBF9901A0F788C7B19D4
:10162600121673A308DBF9901A2822C2AF1216B25B
:1016360012168C901A00740E121678A374061216DF
:1016460078A37415121678901A0378807B0A1216FE
:1016560077A308DBF9901A0F788C7B19121677A3FB
:1016660008DBF91216C51216A3901A2822E493F67F
:1016760022E6438F01538FFD75EF0275B7A575B747
:10168600F1F0538FFE22438F02438F0175EF0275EF
:10169600B7A575B7F1901A0DF0538FFC22901A0D6D
:1016A600745AD178901A0E74A5D178227A3079D0EE
:1016B6007820901A40D173E520F709A3DAF7227A49
:1016C6003079D0901A40E7D17809A3DAF922AB74C1
:1016D600A875BB01027984BB02027985BB03027936
:1016E60086BB04027992BB05027987BB060279A301
:1016F600BB0702799CBB08027988BB09027989E895
:10170600F7227C05120606DCFB22C2AF1206161271
:10171600061D12062412062B1205F71206161206CD
:101726001D12062412062B1205F712061612061DA6
:1017360012062412062BD2AF22C2AF12062B1206B5
:101746002412061D1206161205F712062B1206247F
:1017560012061D1206161205F712062B1206241281
:10176600061D120616D2AF22AE74AF75C2AF1206B0
:10177600161206161206161205F7DEF212062B12BE
:1017860005F7DFF8D2AF22F110F108F10875740100
:10179600757501757600F16E7C05AD5C120606C3A3
:1017A600ED955C70F5C3E55C9401400AC3E55C9475
:1017B600FF40320217C9D1D4D131F110C2AF75EF53
:1017C60012F108DCD50576C3E5769403500280C68F
:1017D600F1080575E5741490009F93F808C3E57544
:1017E60098500280AEF108F1080574C3E574940AB6
:1017F6005002809C120F42D131C2AF75EF12121700
:0118060008D9
:0319FD000210983D
:101A00000E0615FFFFFFFF03040A0301015AA5019B
:101A1000FFFFFFFFFF03FFFFFF25D0FAFA04FF01DE
:091A2000007AFF0101000300FF40
:101A4000234F76736B794D5232304150726F2320A1
:101A500023424C48454C492346333930232020202B
:101A60002020202020202020202020202020202076
:101C0000C2AFC2D353D9BF7581C043B20343FF8073
:101C1000752438752503B1C975EF0275E24043F1AB
:101C20008053A47F75D4FFD2877DFA780379E67C50
:101C300010752200752300901DD67B0675249875BB
:101C400025013087028142208708D8FBD9F9DCF7CB
:101C500081B4308708D8FBD9F9DCF781B4B189E4C5
:101C600093A3C39A6004DDC381B4DBDBB17B600264
:101C7000812B7B08E493FAA3B15CDBF87A30B15C8A
:101C8000752200752300B17BEAFCEBFDC3ED94FEE9
:101C9000400EB17B8A278B28ED30E0048A828B834B
:101CA000B17B7AC270D8C3ED94FE601350CEBD00F4
:101CB00025EC60097520007521FF0200008100A855
:101CC00027A9280809D804D90281D3B17FEA89AAB3
:101CD000F281C50D81A0C3ED94035049EDA2E092BD
:101CE000007AC5C3E5829400E583941C50902000DF
:101CF00010438F02438F0175B7A575B7F1F030001F
:101D00001FA827A9280809438F01538FFDD804D99C
:101D100002A12089AAE275B7A575B7F1F0A3A10DBC
:101D2000538FFC817C7AC1BD030CE493A3FAB140CC
:101D3000DCF8B138817C817EAA22AB23B15CEBFA5E
:101D4000EA6222752608C3E52313F523E52213F57D
:101D50002250066323A0632201D526EAB1C9B1C986
:101D600075260AEAF4200102D287300102C287B147
:101D7000C9C3134002C201D526EB22B17FEAFB2082
:101D80008702A17F308702A184752608AE24AF2583
:101D9000C3EF13FFEE13FEB1CDB1C9C3EA13308711
:101DA000024480FA30E703632201C3E52313F523DD
:101DB000E52213F52250066323A0632201D526D91C
:101DC000E52265236523F52222AE24AF250E0FDE22
:101DD000FEDFFCD20122424C48656C693437316326
:041DE000F390060175
:00000001FF
